:020000040000FA
:10000000031383161330860080309F0093019417EA
:1000100003138312061E0A2806118611B001B101CE
:10002000B6010830940094160615C720061CE72078
:1000300016280130B9003230BA006820B2013B08FE
:10004000B300F030B4000230B9003230BA005420AE
:100050003B08031930283B08B9003C08BA0054207B
:10006000FA30B400B90154200800B3010130B900DE
:10007000B2013230BA006820320803195328B201A5
:10008000F030B4000230B9003230BA0068203308D2
:1000900003194F283308B9003C08BA006820F23031
:1000A000B400B901542008003908BD003A08BE0068
:1000B0000130B9003430BA00363084203D080319CD
:1000C00067283D08B9003E08BA0034308420080093
:1000D0003908BD003A08BE000130B9003430BA001A
:1000E000363084203D08031983283D08B900353097
:1000F000B7208F203E08840039089A208000840AA7
:10010000B90B7C28BF200800B7208F203A08840054
:1001100000088F20840AB90B8828BF2008008C11A2
:1001200093000313831614189328031383128C1D52
:1001300097280800BD008C11031383169115031333
:1001400083128C1DA1281308BE003D08013C031832
:10015000AD28031383169112B0280313831691164A
:100160001116111AB128031383123E080800031355
:10017000831611141118BA280313831208000313ED
:10018000831611151119C228031383120800D030E9
:10019000B4000130B9002030BA00A0015420D130A1
:1001A000B4000130B9008030A0005420D830B40031
:1001B0000130B9000230A0005420F330B400023006
:1001C000B9009730A0000B30A10054200800F43093
:1001D000B4000230B9003F30BA006820401FF12857
:1001E000C7203F1DF4280022BF1D1429361C0A29F0
:1001F000D130B4000130B9003730BA00542040305B
:10020000B4000330B4070130B9002030BA006820D0
:10021000361014294030B4000330B4070130B9005F
:100220002030BA006820AF21BF1E40294030B40002
:100230000530B4070130B9002030BA00682005301D
:10024000B4002030BC00352083132030B3072030A9
:10025000BE0033083E0203183F293E088400000810
:10026000BD00A0308400300884073D088000B00A3B
:1002700050303002031C3D29B001BE0A2929D0218B
:100280003F1E4C294030B4000430B4070130B9009F
:100290002030BA006820D0213F1F60294030B400D0
:1002A0000630B4070130B9002030BA006820403071
:1002B000B4000630B4070130B9000130A00054206A
:1002C000BF1F74294030B4000730B4070130B900B3
:1002D0002030BA0068204030B4000730B407013045
:1002E000B9000130A0005420401C88294030B400DF
:1002F0000830B4070130B9002030BA00682040301F
:10030000B4000830B4070130B9000130A000542017
:10031000C01C9C294030B4000930B4070130B9003A
:100320002030BA0068204030B4000930B4070130F2
:10033000B9000130A000542008000130B90001309C
:10034000A0002030BA004030B4000330B40754207D
:100350000130B9004030B4000230B4070800033067
:10036000B4003508031DB729BB011920CF29350872
:10037000BD003508083C0318BF290830BD003D0802
:10038000BB002030BC0020308400FC218000B5037D
:10039000C10A0319C20A840ABD0BC5291920080025
:1003A0000430B4000130B9002030BA0068202008C1
:1003B000031DFB298313BE0108303E020318F429F4
:1003C00031088400A03084070008BD003E08840086
:1003D000203084073D088000B10A50303102031CF0
:1003E000F229B101BE0ADC290430B4003E08BB008A
:1003F0002030BC001920080042088A004108820011
:100400004030B4000230B4070130B9002030BA00E7
:100410006820A01EC52B0230B4002830BC00352057
:10042000F130B400B9015420F230B400B9015420C5
:100430000330B400B9015420F130B400B9015420A4
:10044000A8132808031DAE2A2908031D322A0330E9
:10045000B4000230BB002030BC000130A000A1017C
:100460001920C72B01302902031D372AC623033068
:100470002902031D3C2AC62B05302902031D492AE7
:100480002A08B700B7170330B400BB01192036148F
:10049000C72B06302902031D902A2F080319522A60
:1004A000FF30AE0001302B02031D5B2A0330C20077
:1004B000C830C100852A02302B02031D6E2A03308A
:1004C000C200DA30C1000230C1070318C20AFC21A1
:1004D000B5000330C200DA30C100872A03302B0296
:1004E000031D8F2A2A08031D7A2A0430C200043013
:1004F000C100852A01302A02031D832A0330C2006D
:10050000FA30C100852AB501C72BFC21B50035089A
:100510002E0203188D2A2E08B500AF21C72BC62B3B
:1005200008302902031D9C2A0330B4000130BB00AF
:100530003830BC001920C72B09302902031DAD2A11
:100540002A08B8000330B400BB0119203808031989
:10055000AB2A8615AC2A8611C72BC62B0130280280
:10056000031DEC2A2908031DBF2A0330B400023002
:10057000BB002030BC00A001A1011920C72B0B300B
:100580002902031DD62A2D08031DD42A2C08031D79
:10059000D42A2B08031DD42A2A08031DD42A033089
:1005A000B400BB011920D52AC62BC72B0A3029025B
:1005B000031DEB2A2D08031DE92A2C08031DE92A37
:1005C0000330B4000130BB002030BC00A001192072
:1005D000EA2AC62BC72BC62B02302802031D7F2B0D
:1005E00001302902031DF52AF92A03302902031DCF
:1005F0003D2B2B08031D392B2A08031D392B0130F5
:100600002902031D052BA001072B0130A00040305B
:10061000B4000130B9002030BA0001302C02031DB3
:10062000142B0530B4073B2B81302C02031D1B2BF0
:100630000430B4073B2B02302C02031D222B063062
:10064000B4073B2B82302C02031D292B0730B40743
:100650003B2B03302C02031D302B0830B4073B2BFF
:1006600083302C02031D372B0930B4073B2BC62BDC
:100670003A2BC62BC72B5420C72B2908031D7E2BD2
:100680008030B4000130B9002030BA0001302C02B3
:10069000031D4D2B0530B407712B81302C02031D37
:1006A000542B0430B407712B02302C02031D5B2B3A
:1006B0000630B407712B82302C02031D622B0730E9
:1006C000B407712B03302C02031D692B0830B407CB
:1006D000712B83302C02031D702B0930B407712B52
:1006E000C62BA01D762B0130A000772BA001A10105
:1006F0000330B4000230B9001920C72BC62B40309C
:100700002802031D842B882B42302802031DC32B93
:1007100001302902031DB12B2C08BD000730BD0597
:100720003D0DBD0D3D0DBD0D3D0DBD0DC130BD04DB
:100730003D089F00FF30BD00BD0B9C2B1F151F19EE
:100740009F2B031383161E0803138312A0001E0899
:10075000A1000330B4000230BB002030BC001920DF
:10076000C72B02302902031DC22B0608BD0007302B
:10077000BD052C08BD043D0886000330B400BB0154
:100780001920C72BC62BC62BC62B00009D210800A5
:10079000123401341034013400340034003408348D
:1007A0003334333401340034003400340134003441
:1007B000003401340934023420340034013401346B
:1007C00000348034323409340434003400340234C8
:1007D000FF34FF34FF34003407340534013402346D
:1007E00008340034003407340534813402340834CA
:1007F000003400340A3403345A340034653400348D
:10080000623400347534003404340334093404345D
:02400E00393D3A
:00000001FF
